:020000040000FA
:04000000803106281D
:080008008031732823008C01F4
:100010008E0121009D019E01220091019201930118
:10002000940121008E110E108E100E110C1503304C
:1000300024008C008E012100951380283030AB0005
:100040003030AC003030AD0022000E108E100E119A
:1000500020003210B21032110800BA0030303A02DB
:10006000031D34282014080031303A02031D3A28B9
:100070002014080032303A02031D402820140800E2
:1000800020100800B90023009E019E161E159D0138
:100090001D169D172000390823009B000800200032
:1000A000B80023009E185528512820003808230046
:1000B0009A00080020003710911A371420103718C2
:1000C000201408002300190808002000B60007309B
:1000D0002100950020003608B0003608B100B211AA
:1000E0008B168B1708000B1D7F2820003108031D7D
:1000F0007D28B2153008B1007E28B1030B1109002C
:1001000020000C1987284030422080318928813016
:1001100042204C30803165202000A70122008E153E
:10012000200032165830AE000230AF0022000E140C
:100130008E140E1520009530A000E930A1002E305D
:10014000A2008031A20BA2288031A10B9F28803110
:10015000A00B9D280000000000000000000022000D
:100160000E1020007F30A000CD30A1001E30A20074
:100170008031A20BB9288031A10BB6288031A00BA9
:10018000B42800000000000022008E1020007F3004
:10019000A000CD30A1001E30A2008031A20BCE28DD
:1001A0008031A10BCB288031A00BC92800000000B2
:1001B000000022000E1120007F30A000CD30A100F1
:1001C0001E30A2008031A20BE3288031A10BE02871
:1001D0008031A00BDE2800000000000022000E1578
:1001E00020007F30A000CD30A1001E30A200803161
:1001F000A20BF8288031A10BF5288031A00BF32841
:1002000000000000000022008E1420007F30A000BB
:10021000CD30A1001E30A2008131A20B0D29813109
:10022000A10B0A298131A00B082900000000000061
:1002300022000E1420007F30A000CD30A1001E301F
:10024000A2008131A20B22298131A10B1F2981310A
:10025000A00B1D2900000000000080311E20593035
:1002600080314F2080315A2020003213201832175D
:100270008131321FB529803162202000A600270875
:100280008131031D4E2921302602031D4929A70A69
:10029000B5294E3080314F208131B5292703031D08
:1002A0006629260880312D202000331120183315AF
:1002B0008131331D5F292608A800A70AB5294E30D1
:1002C00080314F202000A7018131B529023027025B
:1002D000031D7F29260880312D202000331220188D
:1002E00033168131331E78292608A900A70AB529BB
:1002F0004E3080314F202000A7018131B5290330D5
:100300002702031D9829260880312D202000331351
:10031000201833178131331F91292608AA00A70A14
:10032000B5294E3080314F202000A7018131B529F9
:1003300004302702031DB52923302602031DB029EE
:100340002808AB002908AC002A08AD005830AE00E0
:100350000230AF00A701593080314F208131B529DB
:100360004E3080314F202000A70181312000B21D86
:100370003229AE032E0A0319AF032E082F04031DE2
:10038000C82980311E2058302000AE000230AF0056
:1003900030302B028131031DCF293210E129313059
:1003A0002B02031DD5293214E12932302B02031D03
:1003B000DF29321CDD293210DE293214E129803197
:1003C0001E20813120003218E82922000E10EA296F
:1003D00022000E14303020002C02031DF229B2102E
:1003E0008231062A31302C02031DF929B2148231E0
:1003F000062A32302C028231031D042AB21C022A42
:10040000B210032AB214062A80311E208231200045
:10041000B2180D2A22008E100F2A22008E143030BE
:1004200020002D02031D162A3211282A31302D02F8
:10043000031D1C2A3215282A32302D02031D262ABC
:10044000321D242A3211252A3215282A80311E20F5
:100450008231200032192F2A22000E11312A220067
:100460000E152000321A372A22008E11392A220056
:100470008E152000321E3E2A32123F2A3216B21149
:04048000813132296B
:020000040001F9
:02000E00E23FCF
:02001000FF1ED1
:00000001FF
